:100000000C9471080C9491080C9491080C9491082C
:100010000C9491080C9491080C9491080C949108FC
:100020000C9491080C9491080C9491080C949108EC
:100030000C9491080C9491080C9491080C949108DC
:100040000C9491080C9461130C9491080C949108F1
:100050000C9491080C9491080C9491080C949108BC
:100060000C9491080C94952B0C94612B0C94910892
:100070000C9491080C94A2080C9491080C9491088B
:100080000C9491080C9491080C9491080C9491088C
:100090000C9491080C9491080C9491080C9491087C
:1000A0000C9491080C9491080C9491080C9491086C
:1000B0000C9491080C9491080C9491080C9491085C
:1000C0000C9491080C9491080C9491080A73772071
:1000D000310A000A737720300A00414D433A206EFE
:1000E0006F77204D300A00414D433A206E6F7720E4
:1000F0004D310A00414D433A2068616E646C6520C1
:10010000636C6F7365640A00414D433A204D3120A2
:1001100068616E646C652073746174757320636FBD
:100120007272656374696F6E0A00414D433A206EC6
:100130006F77204D320A00414D433A2068616E646A
:100140006C65206F70656E65640A00414D433A200E
:100150006E6F77204D330A00414D433A2068616E3F
:10016000646C65206F70656E65640A00414D433AAA
:10017000206E6F77204D340A00414D433A2068616C
:100180006E646C65206F70656E65640A00414D4356
:100190003A204D342068616E646C6520737461741C
:1001A000757320636F7272656374696F6E0A0041C4
:1001B0004D433A206E6F77204D350A00414D433A4A
:1001C0002068616E646C6520636C6F7365640A00FF
:1001D000414D433A206E6F77204D360A000A414D5B
:1001E00043206873776170206F75743A20000A535A
:1001F0004953383330300A004275696C742077698E
:100200007468204156522D4743433A2000342E361D
:100210002E320020616E64204156522D4C494243DB
:100220003A2000312E382E30002072656C656173E3
:10023000653A20003230313131323238000A6F6E87
:1002400020004A756E203139203230313400202FA1
:10025000200030393A32383A3431000A0A00414D30
:1002600043207374617475733A204D000A00525430
:100270004D207374617475733A204D000A0A002092
:10028000436F6D6D616E646C6973743A0A205354E8
:100290004154202D204669726D7761726520526548
:1002A000766973696F6E2C205374617475732C209A
:1002B0006574632E2E2E0A2048454C50202D207444
:1002C00068697320706167650A002072746D207A16
:1002D0006F6E65333A200020616D63207A6F6E6522
:1002E000333A20002072746D206D617463683A2087
:1002F000002072746D20636C6F7365640A00207255
:10030000746D206F70656E65640A002072746D20D4
:100310006F70656E65640A002072746D206F706581
:100320006E65640A002072746D206F70656E65647E
:100330003A2000505752202B3132563A2000206D7F
:10034000560A4420202B332E33563A202000206DAD
:10035000560A4420202B312E30563A202000206DA2
:10036000560A4420202B312E38563A2020002045B2
:1003700072617375726520454550524F4D202E2E87
:100380002E2000205772697465204144353333387C
:100390003A200020526561642041443533333800EF
:1003A00069326320627573206572726F720A00751C
:1003B0006E6B6E6F776E2069326320737461746543
:1003C0002000657272207374613A20006572722099
:1003D000736C613A2000657272206474613A200087
:1003E0000A0A5349533833303020646562756720F8
:1003F00070726F6D70740A000A0A626F6F747661B2
:100400006C7565203D20000A000A00574454435390
:10041000523A20000A004D4D432046573A20000A28
:100420004275696C742077697468204156522D4773
:1004300043433A2000342E362E320020616E642071
:100440004156522D4C4942433A2000312E382E302D
:10045000002072656C656173653A2000323031317D
:1004600031323238000A6F6E20004A756E20313901
:10047000203230313400202F200030393A32383ADF
:100480003433000A004D435553523A20000A00729B
:1004900065737461727420616674657220636F6C39
:1004A000642072657365740A004D4F44535441547F
:1004B000455F504F5745524544202D3E204D4F44F7
:1004C00053544154455F574149545F524553455435
:1004D00020000D0A004D4F4453544154455F57418D
:1004E00049545F5245534554202D3E204D4F4453AF
:1004F000544154455F574149545F465047415F441A
:100500004F4E4520000D0A004D4F44535441544571
:100510005F574149545F465047415F444F4E452025
:100520002D3E204D4F4453544154455F4650474162
:100530005F52445920000D0A004D4F44535441541A
:10054000455F465047415F52445920000D0A0070F4
:100550008A728E9290748C76989C9AA0A4889E86BB
:100560008478947A9682807C7EA2070051013100C3
:100570000006C10003540201FF7F00703F00000429
:100580000000620200040CC0077FEFABFF00F7F22F
:10059000E9A2A7AB0202000000C6442B312E385658
:1005A00000000000000000000000060051013100C2
:1005B0000005C10003540201FF7F00703F000004EA
:1005C0000000620200040CC0077FEFABFF008E84C6
:1005D0007A42484D0202000000C6442B312E3056AC
:1005E0000000000000000000000002005101300087
:1005F0000001C10003550101FF7F00703F00800131
:100600000000010600040C00001946007DC9555089
:100610004600050A0505000000C574465047410024
:100620000000000000000000000000005112150052
:1006300000002B000000C00000CA5349533833307B
:100640003052544D00005112120000002B000000E7
:10065000C10000C753495338333030020051012FD5
:10066000000008C00003540101FF7F00703F0080BC
:10067000010000010600040C00001946007DC95568
:10068000463C00050A0505000000C47452544D00A4
:1006900000000000000000000000000100510135D2
:1006A000000007C0000340F26F07000000070000D1
:1006B000000000000000000000000000000000003A
:1006C00000000000000000000000CA486F7453776B
:1006D000617052544D0000000000000500510131CE
:1006E000000004C10003540201FF7F00703F0000BE
:1006F000040000A10200040CC0077FEFABFF00F76D
:10070000F2E9A2A7AB0202000000C6442B332E334D
:1007100056000000000000000000000400510132FB
:10072000000003C10003540201FF7F00703F00007E
:10073000040000360200040CD0077FEFABFF00F787
:10074000F2E9A2A7AB0202000000C75057522B31BA
:10075000325600000000000000000003005101318B
:10076000000002C10003540101FF7FFF7F3F0080B2
:10077000010000010600040C0000193C3278E75526
:10078000463C00050A0505000000C674506F7765F9
:100790007200000000000000000000010051013262
:1007A000000000C1000340F26F07000000070000D6
:1007B0000000000000000000000000000000000039
:1007C00000000000000000000000C7486F7453776D
:1007D000617000000000000000000070726F633A5A
:1007E000204E4554464E5F4150503A20434D445FA1
:1007F0004745545F4445564943455F49440A0070A4
:10080000726F633A204E4554464E5F53454E535FD8
:100810004556454E543A20434D445F5345545F4539
:1008200056454E545F52454345495645520A00705D
:10083000726F633A204E4554464E5F53454E535FA8
:100840004556454E543A20434D445F4745545F4515
:1008500056454E545F52454345495645520A00702D
:10086000726F633A204E4554464E5F53454E535F78
:100870004556454E543A20434D445F504C415446F2
:100880004F524D5F4556454E540A0070726F633AA1
:10089000204E4554464E5F53454E535F4556454E98
:1008A000543A20434D445F4745545F4445564943BD
:1008B000455F5344525F494E464F0A0070726F6362
:1008C0003A204E4554464E5F53454E535F4556457C
:1008D0004E543A20434D445F4745545F4445564982
:1008E00043455F5344520A0070726F633A204E458D
:1008F00054464E5F53454E535F4556454E543A203D
:10090000434D445F5245535F4445564943455F5309
:1009100044525F5245500A0070726F633A204E4550
:1009200054464E5F53454E535F4556454E543A200C
:10093000434D445F4745545F53454E534F525F52BA
:10094000454144494E470A0070726F633A204E4554
:1009500054464E5F53454E535F4556454E543A20DC
:10096000434D445F4745545F53454E534F525F5488
:1009700048524553484F4C44530A0070726F633AD3
:10098000204E4554464E5F53454E535F4556454EA7
:10099000543A20756E6B6E6F776E3A200070726FEE
:1009A000633A204E4554464E5F53544F524147459B
:1009B0003A20434D445F4745545F4652555F494E88
:1009C000565F415245415F494E464F0A0070726F73
:1009D000633A204E4554464E5F53544F524147456B
:1009E0003A20434D445F524541445F4652555F446F
:1009F0004154413A2000414D430A0052544D0A00EF
:100A000070726F633A204E4554464E5F53544F52B6
:100A10004147453A20434D445F57524954455F464C
:100A200052555F444154413A2000414D430A00521F
:100A3000544D200070726F633A204E4554464E5F0D
:100A40005049434D473A20434D445F4745545F501A
:100A500049434D475F50524F50530A0070726F63C5
:100A60003A204E4554464E5F5049434D473A204345
:100A70004D445F4652555F434F4E54524F4C3A20BF
:100A800000414D430A0052544D0A0070726F633AA0
:100A9000204E4554464E5F5049434D473A20434D02
:100AA000445F4745545F4652555F4C45445F505242
:100AB0004F50530A0070726F633A204E4554464EB1
:100AC0005F5049434D473A20434D445F4745545F8B
:100AD0004C45445F434F4C4F525F43415041420AA3
:100AE0000070726F633A204E4554464E5F50494342
:100AF0004D473A20434D445F5345545F4652555F3E
:100B00004C45445F53544154450A0070726F633A38
:100B1000204E4554464E5F5049434D473A20434D81
:100B2000445F4745545F4652555F4C45445F5354BC
:100B30004154450A0070726F633A204E4554464E48
:100B40005F5049434D473A20434D445F4745545F0A
:100B50004652555F4C45445F53544154452065729D
:100B6000723A000A0070726F633A204E4554464E46
:100B70005F5049434D473A20434D445F4745545FDA
:100B80004445565F4C4F4341545F5245435F49448F
:100B90000A0070726F633A204E4554464E5F5049CA
:100BA000434D473A20434D445F4652555F434F4EB5
:100BB00054524F4C5F43415041420A0070726F6380
:100BC0003A204E4554464E5F5049434D473A2043E4
:100BD0004D445F5345545F414D435F504F52545F06
:100BE00053544154450A0070726F633A204E455485
:100BF000464E5F5049434D473A20434D445F474579
:100C0000545F414D435F504F52545F5354415445DC
:100C10000A0070726F633A204E4554464E5F504949
:100C2000434D473A20434D445F4745545F434C4F43
:100C3000434B5F53544154450A0070726F633A202E
:100C40004E4554464E5F5049434D473A20434D442C
:100C50005F5345545F4652555F4143544956415492
:100C6000494F4E0A0070726F633A204E4554464E0B
:100C70005F5049434D473A20434D445F5345545FCD
:100C8000504F5745525F4C4556454C0A0070726FA5
:100C9000633A204E4554464E5F5049434D473A20F3
:100CA000756E6B6E6F776E0A0070726F633A204ECE
:100CB0004554464E5F56454E444F523A20434D44AC
:100CC0005F524541445F52544D5F45450A00707282
:100CD0006F633A204E4554464E5F56454E444F5240
:100CE0003A20434D445F57524954455F52544D5F3B
:100CF00045450A0070726F633A204E4554464E5F78
:100D000056454E444F523A20434D445F4D4F44495F
:100D100046595F52544D5F45455F57500A00707207
:100D20006F633A204E4554464E5F56454E444F52EF
:100D30003A20434D445F5345545F464C4153485F0E
:100D4000424F4F545F5245560A0070726F633A200B
:100D50004E4554464E5F56454E444F523A20434D01
:100D6000445F52455345545F465047410A007072F4
:100D70006F633A204E4554464E5F56454E444F529F
:100D80003A20434D445F4745545F4649524D575FB3
:100D900056455253494F4E0A0070726F633A204EC7
:100DA0004554464E5F56454E444F523A20434D44BB
:100DB0005F4745545F754457435F4441435F564125
:100DC0004C55450A0070726F633A204E4554464EAA
:100DD0005F56454E444F523A20434D445F5345546D
:100DE0005F754457435F4441435F56414C55450A44
:100DF0000070726F633A204E4554464E5F56454E22
:100E0000444F523A20434D445F524541445F52544F
:100E10004D5F54454D505F56414C55450A00707228
:100E20006F633A204E4554464E5F56454E444F52EE
:100E30003A20434D445F5345545F52544D5F5445EF
:100E40004D505F504F494E0A0070726F633A204E0A
:100E50004554464E5F56454E444F523A20464F4FFA
:100E6000200A0052544D3A206E6F77204D300A0010
:100E700052544D204D61736B3A200052544D3A202C
:100E80004552524F523A20493243206275732053E3
:100E9000444120737475636B206C6F770A00525461
:100EA0004D3A20636F6D7061746962696C69747921
:100EB00020636865636B3A20006D730A0052544DDD
:100EC0003A206E6F77204D310A00636F6D702E20CF
:100ED000636865636B3A20737563636573730A00B7
:100EE000636F6D702E20636865636B3A206E6F20B0
:100EF0006D61746368657320666F756E640A005275
:100F0000544D204D61736B3A20000A0052544D3A03
:100F10002068616E646C6520636C6F7365642C205F
:100F2000656467650A0052544D3A2068616E646CCE
:100F30006520636C6F7365642C204D30206C657682
:100F4000656C0A0052544D3A206D6F64756C6520D3
:100F500072656D6F7665640A0052544D3A206E6F6B
:100F600077204D320A0052544D204D61736B3A2068
:100F70000052544D3A2068616E646C65206F706554
:100F80006E65640A0052544D3A206D6F64756C654D
:100F90002072656D6F7665640A0052544D3A206E7A
:100FA0006F77204D330A0052544D3A206E6F7720F0
:100FB0004D340A0052544D204D61736B3A2000525B
:100FC000544D3A205365747570204457435F444133
:100FD0004320746F203256350A0052544D3A20682F
:100FE000616E646C65206F70656E65640A005254B2
:100FF0004D3A206D6F64756C652072656D6F766516
:10100000640A0052544D3A20536574646F776E2021
:101010004457435F4441430A0052544D3A206E6F97
:1010200077204D350A0052544D204D61736B3A20A4
:101030000052544D3A20536574646F776E204457C4
:10104000435F4441430A0052544D3A206D6F64752A
:101050006C652072656D6F7665640A0052544D3A76
:10106000206E6F77204D360A0052544D204D61732B
:101070006B3A200052544D3A206D6F64756C6520B8
:1010800072656D6F7665640A000A616D6320776929
:1010900074686F7574207A33207265636F7264733D
:1010A0000A000A72746D20776974686F7574207A0B
:1010B00033207265636F7264730A000A666F722070
:1010C000616D633A2000666F722072746D3A200081
:1010D0000A52544D206873776170206F75743A20FE
:1010E000000011241FBECFEFD1E2DEBFCDBF13E061
:1010F000A0E0B2E0EEE6FFE500E00BBF02C0079023
:101100000D92A03DB107D9F71BBE17E0A0EDB3E0EB
:1011100001C01D92AA33B107E1F70E947D2C0C9407
:10112000B52F0C94000010920E0410927C0087ECF6
:1011300080937A0080917A0084FFFCCF8FEC8093BB
:101140007A0008951F920F920FB60F920BB60F926E
:1011500011242F934F935F936F937F938F939F935C
:10116000AF93BF93EF93FF938091780090917900B4
:10117000A0E0B0E04091D0035091D1036091D20340
:101180007091D303840F951FA61FB71F8093D003C0
:101190009093D103A093D203B093D3032091D403AF
:1011A0002F5F2093D4032223E9F420910E04E22F31
:1011B000F0E0EE0FFF1FEA5FFB4F892F9A2FAB2F56
:1011C000BB27918380831092D0031092D103109299
:1011D000D2031092D303822F8F5F837080930E040B
:1011E00080937C008FEC80937A00FF91EF91BF9108
:1011F000AF919F918F917F916F915F914F912F91BF
:101200000F900BBE0F900FBE0F901F901895E82FF8
:10121000F0E0E370F070EE0FFF1FEA5FFB4F80819C
:10122000918108951F93CF93DF93CDB7DEB7C35459
:10123000D0400FB6F894DEBF0FBECDBF182F8DED96
:1012400091E00E94CF2B812F0E94482C80E092E0F9
:101250000E94BD2B809113068C8380E18D83809149
:10126000C8058F838091120688878C5F8093120651
:1012700082E0898784E08A8782EF8B871C868FE6ED
:101280008D871E878BE08B83CE0101960E941914F7
:1012900081E08A83CE0101960E94DB101093020246
:1012A000CD5BDF4F0FB6F894DEBF0FBECDBFDF9131
:1012B000CF911F910895CF9380E80E94CE2AC82F26
:1012C00080910402809303028091DB0380930402E7
:1012D0008091DC03C81749F0CC2319F08CEC90E026
:1012E00002C083ED90E00E94CF2B80E80E94CE2ABE
:1012F0009091DA03882319F09D7F916002C092607B
:101300009E7F9093DA0380910402833009F482C0B7
:10131000843040F490910302813071F1823008F002
:1013200058C00AC0853009F4D3C0853008F498C08D
:10133000863009F00DC1F0C0992309F406C18AED89
:1013400090E00E94CF2B80E060E041E050E00E94FE
:10135000191181E060E041E050E00E94191182E043
:1013600060E043E050E00E94191182E060E040E05C
:1013700050E00E941911E9C0913051F080E060E026
:1013800041E050E00E94191187EE90E00E94CF2BBF
:101390008091DC03C81771F0CC2361F0C093DC03AB
:1013A00084EF90E00E94CF2B80E00E94120982E03F
:1013B0008093DB038091DC03C81709F445C0CC237C
:1013C00009F042C01092DC0388E091E00E94CF2B2C
:1013D0003BC0923021F08AE291E00E94CF2B8091B5
:1013E000DC03C81771F0CC2361F41092DC0387E3AF
:1013F00091E00E94CF2B81E00E94120981E080934E
:10140000DB038091D903882309F4A2C01092D90389
:1014100083E09CC080910302833021F08BE491E053
:101420000E94CF2B8091DC03C81771F0CC2361F4AC
:101430001092DC0388E591E00E94CF2B81E00E94AE
:10144000120981E08093DB038091D803882309F49B
:101450007FC01092D80381E08093C70584E076C0F6
:1014600080910302843021F08CE691E00E94CF2B22
:101470008091DC03C81781F0CC2371F41092DC0357
:1014800089E791E00E94CF2B81E00E94120985E05C
:101490008093DB031092BF058091DC03C81741F0F5
:1014A000CC2331F0C093DC038DE891E00E94CF2B78
:1014B0008091D603882309F44BC01092D60387E0AD
:1014C0008093C70586E08093DB031092BF0540C080
:1014D00080910302853021F08FEA91E00E94CF2BAA
:1014E0008091DC03C81771F0CC2361F0C093DC035A
:1014F0008CEB91E00E94CF2B80E00E94120984E0E7
:101500008093DB038091D703882379F01092D7036F
:1015100086E08093DB0309C080910302863029F0C6
:101520000D9A80ED91E00E94CF2B8091D603882305
:1015300029F01092D60387E08093C7058091C705F4
:10154000882331F482E00E94120981E08093DB035A
:101550008091D503882331F0809102020E94120904
:101560001092D503CF91089580910402089580913F
:10157000DA03089581E08093D903089581E0809390
:10158000D8031092D7031092D603089581E0809378
:10159000D7031092D8031092D603089581E0809368
:1015A000D6031092D7031092D803089581E0809358
:1015B000D50308956F927F928F929F92AF92BF92C0
:1015C000CF92DF92EF92FF920F931F93CF93DF930F
:1015D000CDB7DEB7C850D1400FB6F894DEBF0FBE0E
:1015E000CDBF4C01E62E3A01FC011082CE010196DE
:1015F00060E070E048E050E00E94852FFE013196E7
:1016000097E080E02191820F9150E1F781959885D4
:10161000891709F059C00E8110E093E0000F111FE7
:101620009A95E1F70115110509F450C089E0A82E3B
:10163000B12CAC0EBD1EB80160507040CE010196B9
:1016400045E050E00E94852F8A819981890FFB80B7
:101650008F0D9C81890F81959D818917C9F5CF2CAC
:10166000DD240B5F1F4FB80160507040C501A6011B
:101670000E94852F20E030E006C08A0D9B1DFC01F2
:101680008081280F3F5F832F90E08C159D05A8F384
:1016900021958C812817F1F48C85803379F4F4013D
:1016A00080818F5F80838E1549F46114710431F05D
:1016B000C301B5014F2D50E00E947C2F8A8187FD28
:1016C0000BC00C0D1D1DB7CF82E007C083E005C025
:1016D00084E003C085E001C080E0C85FDE4F0FB644
:1016E000F894DEBF0FBECDBFDF91CF911F910F9158
:1016F000FF90EF90DF90CF90BF90AF909F908F9032
:101700007F906F900895EF92FF920F931F93CF9366
:10171000DF93CDB7DEB728970FB6F894DEBF0FBEC4
:10172000CDBF7C01CE01019660E070E048E050E062
:101730000E94852FFE01319697E080E02191820F73
:101740009150E1F781959885891749F50E8110E050
:1017500023E0000F111F2A95E1F70115110509F18A
:10176000B80160507040CE01019645E050E00E9403
:10177000852F2A819981920F8B81980F3C81930F3D
:1017800091953D81931779F490E00596080F191F04
:1017900027FFE6CFF7011183008380E005C082E0D8
:1017A00003C083E001C084E028960FB6F894DEBF42
:1017B0000FBECDBFDF91CF911F910F91FF90EF90A2
:1017C000089588E193E00E94CF2B80E008958FE791
:1017D00092E00E94CF2B80E00895CF93DF9300D05A
:1017E000CDB7DEB783E993E00E94CF2B8CE061E0B8
:1017F000AE014F5F5F4F0E94B028882329F085E03B
:1018000092E00E94BD2B0AC08DE092E00E94BD2BA9
:1018100089810E94482C8A810E94482C82E192E0B2
:101820000E94BD2B80E00F900F90DF91CF91089523
:10183000CF93DF9300D000D0CDB7DEB719821A82E4
:101840001B821C828CE289838CE18A83A5E4B4E04C
:10185000FE01319680E090E03D91232F20532A3005
:1018600008F027502193019684309105A9F78981CA
:101870008295807F9A819F70892B89838B81829545
:10188000807F9C819F70892B8A8383E893E00E94EC
:10189000CF2B89810E94482C8A810E94482C8CE0A1
:1018A00061E0AE014F5F5F4F0E94D625882319F09B
:1018B00084E192E002C080E292E00E94BD2B80E0D1
:1018C0000F900F900F900F90DF91CF910895CF93CD
:1018D000DF938EE693E00E94CF2BC0E0D0E080E55E
:1018E000BE0140E00E94DC24219682E0C030D8078F
:1018F000B1F78BE292E00E94BD2B80E0DF91CF91A7
:101900000895EF92FF920F931F93CF93DF9300D030
:1019100000D000D0CDB7DEB782E392E00E94BD2BAD
:1019200081E56AEF70E046E050E09E012F5F3F4F97
:101930000E943925882329F084E492E00E94BD2B7F
:1019400010C07E010894E11CF11C00E010E0F701DA
:1019500081917F010E94482C0F5F1F4F06301105B7
:10196000B1F782E192E00E94BD2B80E026960FB68F
:10197000F894DEBF0FBECDBFDF91CF911F910F91C5
:10198000FF90EF900895CF93DF9380E00E940709C6
:10199000EC0183E393E00E94CF2BBE0180E090E056
:1019A00024E63DE84DE050E00E94142F0E94FF2BFA
:1019B00081E00E940709EC018EE393E00E94CF2BA7
:1019C000BE0180E090E022E836E044E050E00E9472
:1019D000142F0E94FF2B82E00E940709EC018EE485
:1019E00093E00E94CF2BBE0180E090E026E536E038
:1019F00040E050E00E94142F0E94FF2B83E00E94E1
:101A00000709EC018EE593E00E94CF2BBE0180E038
:101A100090E020E13AE340E050E00E94142F0E9461
:101A2000FF2B8EE492E00E94BD2B80E0DF91CF91EE
:101A30000895EF92FF920F931F93CF93DF9300D0FF
:101A4000CDB7DEB785E293E00E94CF2BCE010196A1
:101A50000E94DE2290E00E94FF2B03E512E0C80105
:101A60000E94BD2B89819A810E94FF2B22E1E22EE8
:101A700022E0F22EC7010E94BD2BCE0101960E94EA
:101A8000830B90E00E94FF2BC8010E94BD2B89812F
:101A90009A810E94FF2BC7010E94BD2B80E00F900E
:101AA0000F90DF91CF911F910F91FF90EF900895CC
:101AB0008BE093E00E94CF2B86E00E94752080E0AF
:101AC00008958EEF92E00E94CF2B81E00E94752056
:101AD00080E0089581EF92E00E94CF2B80E00E9489
:101AE000752080E0089584EE92E00E94CF2B0E9442
:101AF000F72390E00E94FF2B82E192E00E94BD2B31
:101B000088E00E94752080E00895CF93DF930F92C4
:101B1000CDB7DEB787ED92E00E94CF2BCE010196C4
:101B200060E040E050E00E94DA0A90E00E94FF2B63
:101B300083E592E00E94BD2B898190E00E94FF2BFB
:101B400082E192E00E94BD2B87E00E94752080E038
:101B50000F90DF91CF910895CF93DF930F92CDB780
:101B6000DEB78AEC92E00E94CF2BCE01019660E0B6
:101B700040E050E00E944C2390E00E94FF2B83E560
:101B800092E00E94BD2B898190E00E94FF2B82E1B0
:101B900092E00E94BD2B85E00E94752080E00F90AE
:101BA000DF91CF9108958EEE91E00E94CF2B88EFC8
:101BB00091E00E94CF2B8DE092E00E94CF2B83E139
:101BC00092E00E94CF2B83E292E00E94CF2B89E229
:101BD00092E00E94CF2B84E392E00E94CF2B8DE312
:101BE00092E00E94CF2B82E492E00E94CF2B8EE401
:101BF00092E00E94CF2B82E592E00E94CF2B8BE5F2
:101C000092E00E94CF2B8EE592E00E94CF2B0E94A3
:101C1000B40A90E00E94FF2B8CE692E00E94CF2B4A
:101C20008EE692E00E94CF2B0E945D2090E00E9401
:101C3000FF2B8CE792E00E94CF2B80E0089585E592
:101C400092E00E94BD2B10923F040895CF93DF9342
:101C5000AC01A0E08A2F90E0880F991F880F991F90
:101C6000FC01E154FD4F60817181B0E02B2F30E029
:101C7000FB01E20FF31FE081EE2359F0240F351F23
:101C8000E90128812E272F7511F4BF5FEFCFAF5FD9
:101C9000E1CFBB2349F081549D4FDC011296ED91B9
:101CA000FC911397099501C081E0DF91CF910895D0
:101CB000CF93DF930F92CDB7DEB7CE0101960E948E
:101CC000432B882309F04CC08981883019F08D306E
:101CD00081F510C080913F04882309F441C08150F0
:101CE00080933F0488E00E94242B80E20E94242BF2
:101CF00088E034C08AE00E94242B8DE00E94242BCF
:101D0000E0913F04EE2371F0F0E0E05CFB4F1082C5
:101D100080E494E00E94260E882321F08EE592E074
:101D20000E94BD2B10923F048FE692E00E94BD2BD3
:101D300017C08B31A9F090913F04903270F40E944B
:101D4000242B80913F04E82FF0E0E05CFB4F998169
:101D500090838F5F80933F0403C087E00E94242B11
:101D60000F90DF91CF9108950F931F93CF93DF933F
:101D7000C6E3D0E0CE010E94952F90E08F70907066
:101D800024E630E0829F8001839F100D929F100D0A
:101D90001124CE0101960E94952F90E08F709070D3
:101DA0009C01220F331F53E0880F991F5A95E1F7CA
:101DB000280F391F020F131FCE0102960E94952F84
:101DC0008F709801280F311DC901DF91CF911F91AC
:101DD0000F910895CF92DF92EF92FF920F931F938E
:101DE00086E390E00E94952F90E08F70907024E63B
:101DF00030E0829F6001839FD00C929FD00C112411
:101E0000EE24D7FCE094FE2C87E390E00E94952F0F
:101E100090E08F7090709C01220F331F63E0880F59
:101E2000991F6A95E1F7280F391FC901AA2797FD65
:101E3000A095BA2FC80ED91EEA1EFB1E88E390E0BB
:101E40000E94952F8F70A7019601280F311D411D0B
:101E5000511DDA01C9015A98EFE9FFE03197F1F716
:101E600000C000005A9AE0E2F0E000E010E020E05C
:101E700030E85B98B901A801482359236A237B23E2
:101E8000411551056105710509F05B9AF8945A985E
:101E90005A9A78943695279517950795319749F76B
:101EA0001F910F91FF90EF90DF90CF90089590E2F7
:101EB0009093B8008E7F8093BA001092BD0084E4A6
:101EC0008093BC0010926A04109269040895CF9325
:101ED0008091BC0087FF67C0C091B900C87FC03641
:101EE00061F0C13620F4CC2309F448C051C0C03899
:101EF000D1F0C03A09F04CC02BC01092DF03E09142
:101F0000CD05F091CE0580818068808380818E7FB1
:101F100080838091BB00838381E08093DF0394EC16
:101F20009093BC0012C0E091CD05F091CE05809158
:101F3000DF039091BB00E80FF11D93838F5F8093C7
:101F4000DF0384EC8093BC0081E08093DE032BC030
:101F5000E091CD05F091CE058091DF0382838081F1
:101F60008160808380818F77808384EC8093BC0044
:101F70001092DE038AE080931A0315C080EA93E092
:101F80000E94CF2B8091BC0080698093BC000BC065
:101F90008FEA93E00E94CF2B8C2F0E94482C8FEF6A
:101FA00092E00E94BD2B8091DE03CF910895CF92E5
:101FB000DF92FF920F931F93CF93DF930F92CDB7D2
:101FC000DEB78091DD03882341F490916A0480910B
:101FD0006904981709F053C0E5C08F3F39F484E6CF
:101FE0000E94EF2A8EEF8093DD03DCC08E3F09F064
:101FF00046C080917705882311F14091690450E033
:1020000023E430E0429FC001439F900D529F900D0A
:10201000112485599B4F0E942520909168048917AF
:1020200071F4809169048F5F80936904843011F4A6
:10203000109269041092DD0310927705B3C00E94DC
:10204000FF2A882309F4AEC08091E0038150809379
:10205000E003882321F084E60E94EF2A10C08091DB
:1020600069048F5F80936904843011F410926904CD
:1020700081E093E00E94BD2B1092DD0393C084EABF
:102080008093BC008091BC0087FFFCCF1091B90009
:10209000187F183059F082EC93E00E94CF2B812FEB
:1020A0000E94482C8FEF92E00E94BD2B2091690482
:1020B00030E083E490E0289FF001299FF00D389FE5
:1020C000F00D1124E559FB4F83818093BB0084E818
:1020D0008093BC008091BC0087FFFCCF1091B900B9
:1020E000187F183159F08CEC93E00E94CF2B812F90
:1020F0000E94482C8FEF92E00E94BD2B11E083E4F8
:10210000C82ED12C94E8F92E04E923C0181719F42D
:102110000093BC001DC0E10FF11D83818093BB00C3
:10212000F092BC008091BC0087FFFCCF2091B900E9
:10213000287F283269F086ED93E029830E94CF2B17
:102140002981822F0E94482C8FEF92E00E94BD2BA4
:102150001F5F20916904822F90E08C9DF0018D9D7E
:10216000F00D9C9DF00D1124E559FB4F82818117E4
:1021700068F68181813059F48091DD038E3F79F0DA
:102180008FEF8093DD0383E08093E00308C0822F0C
:102190008F5F80936904843011F41092690484EC99
:1021A0008093BC000F90DF91CF911F910F91FF9012
:1021B000DF90CF90089560916A04462F50E023E4A9
:1021C00030E0429FF001439FF00D529FF00D11242B
:1021D000E559FB4FDC0183E40D9001928150E1F75A
:1021E0006F5F60936A04643011F410926A0480E0B7
:1021F000089591E090937705809368040895DA013B
:10220000A90190E026E130E0829FF001839FF00D6C
:10221000929FF00D1124E858FA4F618710861286BC
:10222000B183A0831282138255834483168217825E
:10223000089590E026E130E0829FD001839FB00DA9
:10224000929FB00D1124A858BA4F6623D1F412966C
:102250008C91129790E0880F991FED91FC91119746
:10226000E80FF91F5183408312968C9112978F5F6C
:1022700012968C9312978430F1F412961C92129756
:10228000089516968C91169790E0880F991F1496D2
:10229000ED91FC911597E80FF91F51834083169635
:1022A0008C9116978F5F16968C931697843019F43D
:1022B00016961C9216970895CF93DF93EA0190E04B
:1022C00026E130E0829FD001839FB00D929FB00D38
:1022D0001124A858BA4F662309F513968C911397C9
:1022E00012969C9112978917D9F190E0880F991F47
:1022F000ED91FC911197E80FF91F808191819983ED
:10230000888313968C9113978F5F13968C931397F2
:10231000843041F513961C92139724C017968C9124
:10232000179716969C9116978917D1F090E0880F11
:10233000991F1496ED91FC911597E80FF91F808174
:1023400091819983888317968C9117978F5F179641
:102350008C931797843031F417961C92179702C00C
:1023600081E001C080E0DF91CF910895EF92FF926C
:102370000F931F93CF93DF9300D0CDB7DEB7F82E26
:10238000282F30E086E190E0289F8001299F100DE2
:10239000389F100D112408581A4FF80180858823A2
:1023A00009F0BCC08285813041F0813068F0823014
:1023B00089F0833009F04BC028C025B1F801918520
:1023C0009095922395B942C085B1F8019185892BEA
:1023D00085B93BC0F8018585882349F095B1818591
:1023E0008095892385B98585815085870BC0F80143
:1023F0008685882339F085B19185892B85B98685B5
:1024000081508687F80186851AC0F8018685882361
:1024100041F085B19185892B85B986858150868764
:102420000CC0F8018585882341F095B181858095A0
:10243000892385B9858581508587F801858588231D
:1024400031F4838585878485868781E08787F801D5
:10245000E784F1E0EF1609F0CEC08F2D61E0AE0108
:102460004F5F5F4F0E945C11882321F5F801E086E1
:1024700049815A81CA019070009711F4108A4BC0AB
:102480009C01215030402A3F310540F482E0F801A0
:10249000808B518B428B538B448B3DC08C3F91057D
:1024A00019F4F801108637C08F3F9105A1F5F801A6
:1024B000E08A31C08F2D60E0AE014F5F5F4F0E9418
:1024C0005C11882341F589819A8190708130910552
:1024D00051F08130910550F08230910551F08330F8
:1024E0009105C9F40FC0F801E28615C0F801128603
:1024F00012C09AE0F80193878AE5848795878687DA
:1025000082E008C09AE5F80193878AE0848795877E
:10251000868783E08287F80117866DC0F80180897D
:10252000813039F0813060F0823081F0833081F584
:1025300019C025B1F80191859095922395B927C0CE
:1025400085B1F8019185892B85B920C0F80184896E
:10255000882341F085B19185892B85B98489815083
:10256000848B0CC0F8018389882341F095B1818563
:102570008095892385B983898150838BF80183896C
:10258000882331F48189838B8289848B81E0858BD8
:10259000F8018589882379F18F2D61E0AE014F5FC5
:1025A0005F4F0E945C11882321F561E0F80160878C
:1025B00049815A81CA019070009711F4108A19C09C
:1025C0009C01215030402A3F310540F482E0F8015F
:1025D000808B518B428B538B448B0BC08C3F91056E
:1025E00019F4F801108605C08F3F910511F4F80128
:1025F000608BF801158A0F900F90DF91CF911F919A
:102600000F91FF90EF900895DB0190E026E130E01C
:10261000829FF001839FF00D929FF00D1124E858E6
:10262000FA4F80858C93828511968C9311978485BF
:1026300012968C931297838513968C9313978089A7
:1026400014968C931497828915968C93159781898B
:1026500016968C9316970895CF92DF92EF92FF9281
:102660000F931F93CF93DF930F92CDB7DEB77B010C
:1026700089830E94062A898181600E94292A8823F1
:1026800021F40E941E2A81E012C081E00E945E2A8D
:10269000182F00E080E00E945E2AC82EDD24C02AA8
:1026A000D12A0E941E2AF701D182C08280E00F90B9
:1026B000DF91CF911F910F91FF90EF90DF90CF901E
:1026C00008951F920F920FB60F920BB60F9211241E
:1026D0002F933F934F935F936F937F938F939F932A
:1026E000AF93BF93EF93FF930E948E2A8091E103F3
:1026F0009091E203A091E303B091E4030196A11D40
:10270000B11D8093E1039093E203A093E303B093A0
:10271000E4038091E5039091E60301969093E6032C
:102720008093E50323E0883E920739F481E08093AB
:10273000BD051092E6031092E5038091E7038F5FD9
:102740008093E703843629F481E08093BE051092DC
:10275000E7038091E8038F5F8093E8038A3071F488
:102760000E94052B81E08093CA051092E8038091B6
:102770000304882319F0815080930304FF91EF91A3
:10278000BF91AF919F918F917F916F915F914F9189
:102790003F912F910F900BBE0F900FBE0F901F9087
:1027A000189585B1817F85B9209A28988FEC97E09C
:1027B0000197F1F700C0000021E0199B20E081E0C3
:1027C0001A9B80E091E01B9B90E0289AEFECF7E0E9
:1027D0003197F1F700C0000063B141E01A9B40E07F
:1027E00031E01B9B30E051E061FF50E0251322E017
:1027F000841382E0931392E0E82FEE0FE80FE20FCC
:1028000089E0989F902D1124E90FF0E0E15BFA4FE9
:102810008491089590E08057904062E070E00E94BB
:102820003F2F862F0895FC018481869586958170BF
:102830000895FC0183819481890F8195858382812C
:10284000DF0123E090E005C015963C911597930FAA
:102850002F5F11962817C0F3DF01A80FB11D9195C6
:1028600013969C9313978F5F82830895CF93DF9382
:10287000EC0188818E7F806888830E94D70F8881D1
:102880008F77888380E0DF91CF910895FC01838169
:102890009481890F819595819817D9F4828190E070
:1028A000019753E040E008C02E0F3F1FD901139657
:1028B0002C911397420F5F5F252F30E028173907BF
:1028C0009CF3E80FF91F41958381841721F082E082
:1028D000089581E0089580E008959F92AF92BF929D
:1028E000CF92DF92EF92FF920F931F93CF93DF93DC
:1028F000CDB7DEB760970FB6F894DEBF0FBECDBF81
:102900008C017B01FE013296ACE5B3E086E00D90D0
:1029100001928150E1F7D80114962C9114972695D5
:1029200026952A3009F447C32B3040F4243009F4AB
:102930004FC0263011F00C94E11F09C02C3209F46D
:102940008FC4203311F00C94E11F0C94281DF80162
:102950008085813011F00C94E11F8BED97E00E948F
:10296000CF2BD80116968C911697F7018383179673
:102970009C91179714968C9114978C5F8C7F292FBC
:102980002370822B84838091C805868314968C9152
:10299000149783709C7F892B878318968C91189746
:1029A00080871186128681E8838782E0848782E7A8
:1029B000858781E586878BE287878DEB808B82E92F
:1029C000818B128A138A83E8848B82E10C94202005
:1029D000D80118968C911897803209F49FC08132E3
:1029E00048F4813009F446C0813088F0823009F023
:1029F000D9C26EC0823209F45EC1823208F4BDC011
:102A0000873209F41AC28D3209F0CCC284C18FEF2B
:102A100097E00E94CF2BF801818580931306828571
:102A2000809314068681D70113968C931397978110
:102A300084818C5F8C7F292F2370822B14968C933A
:102A400014978091C80516968C931697848183708D
:102A50009C7F892B17968C931797808518968C935B
:102A6000189719961C920E94D60A0E94712087E03E
:102A70000C94FA1E8FE298E00E94CF2BD801169694
:102A80008C911697F701838317969C91179714964C
:102A90008C9114978C5F8C7F292F2370822B8483D9
:102AA0008091C805868314968C91149783709C7FBF
:102AB000892B878318968C9118978087118680912F
:102AC0001306828780911406838789E00C94202066
:102AD0008FE598E00E94CF2BD80116968C9116971F
:102AE000F701838317969C91179714968C911497EE
:102AF0008C5F8C7F292F2370822B84838091C80563
:102B0000868314968C91149783709C7F892B87837E
:102B100018968C91189780871186FBC28BE898E0F5
:102B20000E94CF2BD80116968C911697F7018383BC
:102B300017969C91179714968C9114978C5F8C7FA5
:102B4000292F2370822B84838091C8058683149655
:102B50008C91149783709C7F892B878318968C9116
:102B6000808711860E94EE29D7011A968C931A97B6
:102B700081E01B968C931B97CCC08CEB98E00E9455
:102B8000CF2BF8018681D70113968C9313979781E9
:102B900084818C5F8C7F292F2370822B14968C93D9
:102BA00014978091C80516968C931697848183702C
:102BB0009C7F892B17968C931797808518968C93FA
:102BC000189719961C92A384BB24948580E0A82AA8
:102BD000B92AC58496840E94EE290197A816B906E1
:102BE00029F48FEFF7018287838708C0C50101961A
:102BF000D7011A968C931A971B969C93F501EE0FAA
:102C0000FF1FEE59FC4F0C2D10E060817181600FA9
:102C1000711FC7010C96492D50E00E94662FB5E048
:102C2000BC1560F0C801890D911D8530910534F007
:102C3000F701E01BF10B8091C805818BE2E0AE1635
:102C4000B104C8F4FDE0FC1570F1DD24C601890D66
:102C5000911D8D3091053CF1F701EC19FD09809132
:102C6000C80590E08057904062E070E00E943F2FDE
:102C7000605A618F18C049E04C15A8F0DD24C601E8
:102C8000890D911D8930910574F0F701EC19FD094A
:102C90008091C80590E08057904062E070E00E940B
:102CA0003F2F605A658B892D875FD70112968C93D1
:102CB00012970C94042088EE98E00E94CF2BF80124
:102CC0008681D70113968C931397978184818C5FAB
:102CD0008C7F292F2370822B14968C9314978091CC
:102CE000C80516968C931697848183709C7F892BD8
:102CF00017968C931797808518968C93189719962A
:102D00001C92199781E01A968C931A971B961C9225
:102D10001B9789E0CBCF88E199E00E94CF2BF80187
:102D20008681D70113968C931397978184818C5F4A
:102D30008C7F292F2370822B14968C93149780916B
:102D4000C80516968C931697848183709C7F892B77
:102D500017968C931797808518968C9318971996C9
:102D60001C92199781859AE012969C931297843051
:102D7000C9F1853058F4813009F1813098F0823002
:102D800001F1833011F00C9404201EC0863009F448
:102D90003FC08630D8F18730E9F1883011F00C94CB
:102DA000042048C0F701128680EC83870E94B70A8E
:102DB000D7011C968C931C970C9404208091BB0522
:102DC0000AC08091C10515C080E00E940709969550
:102DD000879596958795F701828780E48387148687
:102DE0000C94042081E00E9407099695879596959A
:102DF0008795D7011A968C931A9780E41B968C932B
:102E00001B971C961C921C970C94042082E0DDCF2B
:102E100083E0E9CFF701128680EC83870E9460206F
:102E2000D7011C968C930E946020F70195878BE058
:102E30000C9420208091CC05DCCF88E499E00E949E
:102E4000CF2BF8018681D70113968C931397978126
:102E500084818C5F8C7F292F2370822B14968C9316
:102E600014978091C80516968C9316978481837069
:102E70009C7F892B17968C931797808518968C9337
:102E8000189719961C9219978185843009F43CC0D3
:102E9000853050F48130B9F0813090F08230E9F023
:102EA000833009F07DC026C0863009F441C08630E9
:102EB000A8F1873009F474C0883009F071C042C0AD
:102EC000F7010C941E208FE3D7011A968C931A9762
:102ED000809168039091690309C08FE3D7011A9626
:102EE0008C931A9780916A0390916B03FC01B996B9
:102EF000E49133C08FE3D7011A968C931A9780918F
:102F00006C0390916D03F2CF8FE3D7011A968C93E7
:102F10001A9780916E0390916F03E8CF8FE3D701EA
:102F20001A968C931A978091700390917103DECF5B
:102F30008FE3D7011A968C931A9780917203909120
:102F40007303D4CF8FE3F70182878091760390914A
:102F50007703FC01B996E491D7011B96EC931B977C
:102F6000FC01B896E4911C96EC931C97FC01B79673
:102F7000E4911D96EC931D97FC01B696E4911E9684
:102F8000EC931E97FC01B596E4911F96EC931F9766
:102F90008496FC01849150968C9350978EE086CE57
:102FA000D7011EC48BE799E00E94CF2BF8018085E2
:102FB0000E94482C48C5D80118968C9118978131E9
:102FC00009F452C0823109F4B2C0803109F0F9C766
:102FD0008DE999E0288B0E94CF2BF8018185288903
:102FE000882351F08130D1F4288B0E945D202889FC
:102FF000882311F483ED13C0D7011A961C921A97F7
:1030000082E01B968C931B971C961C921C9719961A
:103010001C92199712962C93129705C089ECF70110
:10302000818787E08283D80116968C911697F701E5
:10303000838317969C91179714968C9114978C5FA5
:103040008C7F292F2370822B84838091C8058683EF
:1030500014968C91149783709C7F892B8783189684
:103060008C9118978087D0C78DEC99E00E94CF2B68
:10307000D80116968C911697F701838317969C9129
:10308000179714968C9114978C5F8C7F292F23703F
:10309000822B84838091C805868314968C91149723
:1030A00083709C7F892B878318968C9118978087D3
:1030B00011861A96AC901A97BB241B969C911B976D
:1030C00080E0A82AB92A1C96CC901C97C286199633
:1030D0008C911997882321F0813009F095C70EC093
:1030E00086EF99E00E94CF2BB50160507040C70178
:1030F0000B964C2D50E00E94852F16C08BEF99E067
:103100000E94CF2B0E945D20882329F483EDF701D4
:10311000818787E095C79701255F3F4F80E5B5011F
:103120004C2D50E00E9481228C2D885FBECD80E026
:103130009AE00E94CF2BF801C280F6EFCF0ED801A3
:103140001A96AC901A97BB241B969C911B9780E013
:10315000A82AB92A19968C911997882321F08130D1
:1031600009F05DC014C08AE29AE00E94CF2BF701FB
:10317000C286B50160507040C8010C964C2D50E0DD
:103180000E949D2FD70119961C92199748C08FE273
:103190009AE00E94CF2B8EE493E00E94BD2BC501E4
:1031A0000E94FF2B84E593E00E94BD2B8C2D90E0C4
:1031B0000E94FF2B8CE493E00E94BD2B0E945D20B7
:1031C000F701882349F1C28611868CE7BE016F5F43
:1031D0007F4F0E94E7208823B1F4698161616F7796
:1031E00069838CE70E940C21882311F0F70114C039
:1031F0009801245F3F4F80E5B5014C2D50E00E94BF
:103200001125882361F0D7011A961C921A9783ED35
:1032100019968C93199703C0128683ED8187D80184
:1032200016968C911697F701838317969C911797A2
:1032300014968C9114978C5F8C7F292F2370822B8E
:1032400084838091C805868314968C91149783702B
:103250009C7F892B878318968C9118978087EFC65F
:10326000D80118968C9118978C3009F468C38D306A
:10327000A8F4853009F4B7C0863030F4882321F1F2
:10328000843009F0C8C357C0873009F4E2C08730E2
:1032900008F4DCC0883009F0BEC361C1893109F48B
:1032A00015C38A3138F48D3009F4C3C2813109F075
:1032B000B2C375C38E3109F406C38D3209F43CC321
:1032C0008A3109F0A8C335C384E39AE00E94CF2B6A
:1032D000F8018681D70113968C9313979781848187
:1032E0008C5F8C7F292F2370822B14968C931497DC
:1032F0008091C80516968C931697848183709C7F65
:10330000892B17968C931797808518968C9318970E
:1033100019961C9219971A961C921A9782E31B967B
:103320008C931B9781E01C968C931C971D961C9286
:103330001D978BE0BBCC8CE59AE00E94CF2BF80167
:103340008681D70113968C931397978184818C5F24
:103350008C7F292F2370822B14968C931497809145
:10336000C80516968C931697848183709C7F892B51
:1033700017968C931797808518968C9318971996A3
:103380001C9219971A961C921A9788E012968C93A1
:1033900012978285882321F0813009F04CC615C030
:1033A00081E89AE00E94CF2BF8018385882321F0E1
:1033B000843009F040C606C01092C70582E30E941F
:1033C000D42A22C60E94CE0A1FC686E89AE00E942E
:1033D000CF2BD8011B968C911B97843009F02BC6FC
:1033E0000E946D2011C68BE89AE00E94CF2BF80155
:1033F0008681D70113968C931397978184818C5F74
:103400008C7F292F2370822B14968C931497809194
:10341000C80516968C931697848183709C7F892BA0
:1034200017968C931797808518968C9318971996F2
:103430001C9219971A961C921A9787E01B968C93E8
:103440001B971C961C921C978AE030CC85EB9AE067
:10345000B6C581EE9AE00E94CF2BF8012485458500
:103460008285882321F0813009F041C227C0C22E15
:10347000DD24942F80E0C82AD92A83858130B1F0D9
:10348000813020F0823009F087C112C080E061E015
:10349000A6010E9419110E94B40A823009F027C2C5
:1034A000CC2009F024C20E94BA0A21C281E001C0E6
:1034B00082E061E0A6010E94191119C2F80183851A
:1034C000813081F0813018F0823049F516C0222316
:1034D00019F02F3F29F402C080E015C080E01AC027
:1034E00080E01BC0222319F02F3F29F402C081E0A5
:1034F0000AC081E00FC081E010C0222319F02F3FE5
:1035000059F407C082E060E040E020E00E942A20F9
:10351000EEC182E061E0F8CF82E062E0F7CFD8014F
:103520008681F701838317969C91179714968C9147
:1035300014978C5F8C7F292F2370822B848380913A
:10354000C805868314968C91149783709C7F892B71
:10355000878318968C91189780878CEC6EC58BE0CA
:103560009BE00E94CF2B19820DC0F801E80FF11DDE
:1035700083810E94482C8AE593E00E94BD2B8981BB
:103580008F5F89838981D80112969C911297891740
:1035900060F38CE493E00E94BD2BF80182858823C0
:1035A00009F023C18385813009F44FC0813020F0B8
:1035B000823009F0E4C08FC080E0BE01685F7F4FB9
:1035C0000E9404138985882319F0813071F404C0A6
:1035D000F701148615860EC08FEFD7011C968C93C9
:1035E0001C971D961C921D9705C08A85F70184873C
:1035F0008B85858781E0D7011E968C931E979CE072
:1036000012969C9312979885913009F0B5C082E08C
:103610001B968C931B978C85882319F0813071F44D
:1036200004C0F7011786108A0EC08FEFD7011F96CE
:103630008C931F9750961C92509705C08D85F7016B
:1036400087878E85808B81E08DC081E0BE01685FB9
:103650007F4F0E9404138985882319F0813071F40B
:1036600008C0D7011C961C921C971D961C921D9792
:103670000EC08FEFF7018487158609C08A85D701B0
:103680001C968C931C978B851D968C931D9782E0BE
:10369000F70186879CE0928398859130C9F48387EF
:1036A0008C85882319F0813049F403C01786108A6D
:1036B00009C08FEFF7018787108A04C08D8587873F
:1036C0008E85808B82E0F701818B8FE082838DC0B5
:1036D00081E083878AC082E0BE01685F7F4F0E94DD
:1036E00004138985882319F0813071F404C0F7012F
:1036F000148615860EC08FEFD7011C968C931C97ED
:103700001D961C921D9705C08A85F70184878B85BD
:10371000858783E0D7011E968C931E978CE01296C6
:103720008C9312978885813031F582E01B968C93BB
:103730001B978C85882319F0813071F404C0F70140
:103740001786108A0EC08FEFD7011F968C931F9794
:1037500050961C92509705C08D85F70187878E85FE
:10376000808B83E0D70151968C9351978FE012960E
:103770008C9312973AC081E0F701838736C085E3C6
:103780009BE00E94CF2BD8011A968C910E94482C66
:1037900083E69BE00E94CF2BF8018681D701139628
:1037A0008C931397978184818C5F8C7F292F237052
:1037B000822B14968C9314978091C80516968C933F
:1037C0001697848183709C7F892B17968C9317970B
:1037D000808518968C9318978CEC19968C93199772
:1037E0001A961C921A9788E061CAF8018681D7015F
:1037F00013968C931397978184818C5F8C7F292FEC
:103800002370822B14968C9314978091C80516967A
:103810008C931697848183709C7F892B17968C9349
:103820001797808518968C93189719961C9219975C
:1038300046C085E69BE00E94CF2BF8018285882355
:1038400019F08130A1F40CC0D7011B961C921B9774
:103850001C961C921C9719961C9219978AE00DC011
:10386000F7018387148611868AE0828308C08CEC76
:10387000D70119968C93199787E012968C93F801CB
:103880008681D70113968C931397978184818C5FDF
:103890008C7F292F2370822B14968C931497809100
:1038A000C80516968C931697848183709C7F892B0C
:1038B00017968C931797808518968C9318971A965D
:1038C0001C921A97A1C382E99BE079C38CEB9BE021
:1038D0000E94CF2BF8018685882319F00E94BE0A2A
:1038E00006C00E94B40A853011F40E94C60AD801AD
:1038F00016968C911697F701838317969C911797CC
:1039000014968C9114978C5F8C7F292F2370822BB7
:1039100084838091C805868314968C911497837054
:103920009C7F892B878318968C91189780871186A6
:1039300085C387EE9BE043C382E19CE040C38AE3FA
:103940009CE00E94CF2BD80116968C911697F70118
:10395000838317969C91179714968C9114978C5F7C
:103960008C7F292F2370822B84838091C8058683C6
:1039700014968C91149783709C7F892B878318965B
:103980008C9118978087128688E082831A968C9192
:103990001A978823A1F1813009F036C3B7C185E6B3
:1039A0009CE00E94CF2BD80116968C911697F701B8
:1039B000838317969C91179714968C9114978C5F1C
:1039C0008C7F292F2370822B84838091C805868366
:1039D00014968C91149783709C7F892B87831896FB
:1039E0008C9118978087128688E082831A968C9132
:1039F0001A97882321F0813009F006C302C08FEFA7
:103A000018C1F8018385882319F00E946520CDC272
:103A10000E946920CAC28DE89CE00E94CF2B1982C7
:103A20000DC0F801E80FF11D83810E94482C8AE542
:103A300093E00E94BD2B89818F5F89838981F80182
:103A40009281891770F38CE493E00E94BD2BB9C278
:103A5000D80118962C911897243009F40EC12530FE
:103A600060F42130E9F0213008F485C1223009F4F6
:103A700068C0233009F0A1C2B2C0273009F4F1C1F7
:103A8000283038F4253009F444C1263009F095C2B5
:103A9000B3C1283009F424C2293009F08EC256C2BD
:103AA00089EA9CE00E94CF2BF801C1849284D384E0
:103AB000A4848681D70113968C9313979781848170
:103AC0008C5F8C7F292F2370822B14968C931497F4
:103AD0008091C80516968C931697848183709C7F7D
:103AE000892B17968C931797808518968C93189727
:103AF00087E012968C93B0E1BA1510F482E85BC2AD
:103B00000E945D20882309F493C0CC2011F490E535
:103B1000C92E692D70E09D2D80E0682B792B9701CF
:103B2000265F3F4F8C2D4A2D50E00E948122882332
:103B300009F0A1C0D70119961C9219978A2D895FA7
:103B4000B5C88EEC9CE00E94CF2BF801C184A28402
:103B5000D38444858681D70113968C9313979781DC
:103B600084818C5F8C7F292F2370822B14968C93F9
:103B700014978091C80516968C931697848183704C
:103B80009C7F892B17968C931797808518968C931A
:103B9000189787E012968C931297413110F082E8C3
:103BA00049C0488B0E945D204889882311F480E831
:103BB00002C2CC2011F480E5C82E6A2D70E09D2D44
:103BC00080E0682B792B9801235F3F4F8C2D50E0CC
:103BD0000E941125882309F499C081E82AC084EF46
:103BE0009CE00E94CF2BD80116968C911697F70176
:103BF000838317969C91179714968C9114978C5FDA
:103C00008C7F292F2370822B84838091C805868323
:103C100014968C91149783709C7F892B87831896B8
:103C20008C91808787E082830E945D20882331F415
:103C300080E8D70119968C931997E6C18CE7BE01ED
:103C40006F5F7F4F0E94E7208823A9F48981982F16
:103C50009161D80119962C911997222311F081694D
:103C600002C0892F8F7789838CE769810E940C219C
:103C7000882309F49AC181E89EC18EE19DE00E94EB
:103C8000CF2BF8018681D70113968C9313979781D8
:103C900084818C5F8C7F292F2370822B14968C93C8
:103CA00014978091C80516968C931697848183701B
:103CB0009C7F892B17968C931797808518968C93E9
:103CC000189787E012968C93129782B18C7F82B9F5
:103CD000818580FD119AF801818581FD109A8FEF11
:103CE0009FE00E94952F8983D80119966C911997AE
:103CF00090E0262F30E08227932783709070009702
:103D000029F063708FEF9FE00E94A72FF7011186C3
:103D10007BC18AE49DE00E94CF2BD80116968C913E
:103D20001697F701838317969C91179714968C9199
:103D300014978C5F8C7F292F2370822B8483809132
:103D4000C805868314968C91149783709C7F892B69
:103D5000878318968C911897808787E08283389A9A
:103D60008FEF99E6A8E181509040A040E1F700C0B4
:103D7000000038981AC18EE69DE00E94CF2BF80112
:103D80008681D70113968C931397978184818C5FDA
:103D90008C7F292F2370822B14968C9314978091FB
:103DA000C80516968C931697848183709C7F892B07
:103DB00017968C931797808518968C93189787E0A1
:103DC00012968C93129719961C92199720E00FC0A7
:103DD000822F90E0F701E80FF91F42E050E04C0F0E
:103DE0005D1F840F951FDC018C9182872F5F25302A
:103DF00078F38CE0F70124C189E99DE00E94CF2B84
:103E0000D80116968C911697F701838317969C918B
:103E1000179714968C9114978C5F8C7F292F2370A1
:103E2000822B84838091C805868314968C91149785
:103E300083709C7F892B878318968C911897808735
:103E400087E082838DEC81878091E903882309F4E0
:103E5000DBC0A701465F5F4F8CE061E00E94B028A5
:103E60006AC085EC9DE0288B0E94CF2BD801199663
:103E70008C91199780931D061A968C911A978093AE
:103E80001E0616968C911697F701838317969C91C0
:103E9000179714968C9114978C5F8C7F392F337001
:103EA000832B84838091C805868314968C91149704
:103EB00083709C7F892B878318968C9118978087B5
:103EC000288922838DEC81878091E903882309F476
:103ED0009BC08CE061E04DE156E00E94D62563C0B6
:103EE00081EF9DE00E94CF2BD80116968C911697FA
:103EF000F701838317969C91179714968C911497CA
:103F00008C5F8C7F292F2370822B84838091C8053E
:103F1000868314968C91149783709C7F892B87835A
:103F200018968C91808787E08283B7016F5E7F4F00
:103F300088E40E9412298823E9F5D70112968C9112
:103F400012978E5F12968C93129730C08EE19EE08E
:103F50000E94CF2BD80119966C91199760931D067A
:103F600016968C911697F701838317969C91179755
:103F700014968C9114978C5F8C7F292F2370822B41
:103F800084838091C805868314968C9114978370DE
:103F90009C7F892B878318968C91808787E082830A
:103FA00088E40E94EB28882329F4D70119961C92F3
:103FB00019972AC08FEFF70126C089E49EE00E947E
:103FC000CF2BD80116968C911697F70183831796FD
:103FD0009C91179714968C9114978C5F8C7F292F46
:103FE0002370822B84838091C805868314968C91DC
:103FF000149783709C7F892B878318968C91808778
:1040000087E0828381EC8187D70111961C921197FA
:1040100081E060960FB6F894DEBF0FBECDBFDF9192
:10402000CF911F910F91FF90EF90DF90CF90BF90B5
:10403000AF909F9008958CECF7018187128688E0FD
:104040008283E2CF8FEC95E00895FC01878186950D
:1040500086950895982F842F913099F0913018F01B
:10406000923051F51CC0609316063AE0632F0E940F
:10407000332F80931C06822F0E94332F80931806C3
:10408000089560931B063AE0632F0E94332F8093BC
:104090002106822F0E94332F80931A060895609381
:1040A00015063AE0632F0E94332F80932006822F5B
:1040B0000E94332F8093320608958091B7030895AC
:1040C0008091F0039091F103089581E08093EF03D4
:1040D000089581E08093EE03089581E08093ED03DD
:1040E000089581E08093EB0308951F93CF93DF93AE
:1040F000CDB7DEB7C354D0400FB6F894DEBF0FBEC5
:10410000CDBF182F80ED90E10E94CF2B812F0E9410
:10411000482C88E793E00E94BD2B809113068C8386
:1041200080E18D838091C8058F83809112068887F6
:104130008C5F8093120682E0898784E08A8782EF11
:104140008B8787E08C878FE68D871E878BE08B833C
:10415000CE0101960E94191481E08A83CE01019656
:104160000E94DB101093B503CD5BDF4F0FB6F894C0
:10417000DEBF0FBECDBFDF91CF911F91089580911B
:104180001706982F917080FD08C08091FC0388234A
:1041900021F01092FC0381E008959093FC0380E0ED
:1041A000089580911706982F917080FF08C0809124
:1041B000FD03813021F081E08093FD030895909309
:1041C000FD0380E0089590911706892308950F93C9
:1041D0001F93CF93DF930F92CDB7DEB78B01898307
:1041E0000E946329898181600E948629882321F4A5
:1041F0000E947B2981E00AC080E00E94BC2989835B
:104200000E947B298981F801808380E00F90DF91F3
:10421000CF911F910F9108951F93CF93DF9300D0FB
:10422000CDB7DEB76A8389830E94632989810E94A2
:1042300086296A81882321F40E947B2981E009C0B4
:10424000862F0E948629182F0E947B2981E0111158
:1042500080E00F900F90DF91CF911F9108951F93F1
:10426000CF93DF930F92CDB7DEB7809116068130E2
:1042700029F08130E0F08230F1F405C01092F403AF
:104280001092F50309C08091F40390911C068917E0
:1042900028F48F5F8093F40311E00EC08091F50342
:1042A0008F5F8093F50390911806891721F410927F
:1042B000F4031092F50310E080911B06813029F081
:1042C0008130F0F0823001F506C01092F6031092B2
:1042D000F703126019C012608091F60390912106D5
:1042E000891720F48F5F8093F6030EC01D7F8091A5
:1042F000F7038F5F8093F70390911A06891721F4D3
:104300001092F6031092F70380911506813029F080
:104310008130F0F0823001F506C01092F80310925F
:10432000F903146019C014608091F803909120067D
:10433000891720F48F5F8093F8030EC01B7F809154
:10434000F9038F5F8093F90390913206891721F466
:104350001092F8031092F9038091B703882311F1AA
:104360008CE7BE016F5F7F4F0E94E7208823D1F466
:1043700081E08093F2038981809317068F6189839E
:1043800010FF02C08D7F898311FF03C089818B7F5D
:10439000898312FF03C08981877F89838CE76981C4
:1043A0000E940C210F90DF91CF911F9108951F93D0
:1043B000CF93DF9300D0CDB7DEB7162F8CE7BE01C9
:1043C0006F5F7F4F4A830E94E7204A81882381F4F0
:1043D000642F61236161409589814823642B69833F
:1043E0008CE70E940C2191E0882319F490E001C031
:1043F00091E0892F0F900F90DF91CF911F91089539
:104400001F93CF93DF930F92CDB7DEB789830E94BE
:10441000632989810E948629882329F089E00E94E6
:104420008629882321F40E947B2981E009C080E04D
:104430000E948629182F0E947B2981E0111180E0BB
:104440000F90DF91CF911F910895CF92DF92EF925D
:10445000FF920F931F93CF93DF930F92CDB7DEB7E9
:10446000F82E8B016A010E9463298F2D0E948629F4
:10447000882379F080E00E948629882351F00E94E9
:104480006E29EE24E394EF288E2D0E94862988233E
:1044900021F40E947B2981E02AC080E00E94BC298F
:1044A00089830E947B298981F80180830E94632986
:1044B0008F2D0E948629882361F081E00E94862941
:1044C000882339F00E946E298E2D0E948629882328
:1044D00021F40E947B2982E00AC080E00E94BC296E
:1044E00089830E947B298981F601808380E00F9077
:1044F000DF91CF911F910F91FF90EF90DF90CF90C0
:104500000895AF92BF92CF92DF92EF92FF920F93F6
:104510001F93CF93DF930F92CDB7DEB7182F062FDF
:104520006A01E22EA32E79830E946329812F880FCE
:104530000E9486297981882391F1872F0E948629FC
:10454000882369F1802F0E948629882341F10E94E7
:104550006E29812F880F81600E9486298823F9F0B7
:104560000E2D1A2DEE24FF2456010894A108B1083F
:104570000FC0EA14FB0411F480E001C081E00E9446
:10458000BC29F80180830894E11CF11C0F5F1F4FC8
:10459000EC14FD0471F70E947B2980E003C00E94A7
:1045A0007B2981E00F90DF91CF911F910F91FF90B8
:1045B000EF90DF90CF90BF90AF900895EF92FF9271
:1045C0000F931F93CF93DF93CDB7DEB728970FB626
:1045D000F894DEBF0FBECDBF7C0180E560E070E0E7
:1045E00048E050E09E012F5F3F4F0E9481228823C8
:1045F00009F044C0FE01319697E02191820F91505D
:10460000E1F781959885891731F08AE793E00E9458
:10461000BD2B82E034C00E8110E083E0000F111F3B
:104620008A95E1F70115110539F180E5B80145E0FA
:1046300050E09E012F5F3F4F0E9481228823F1F4BA
:104640002A819981920F8B81980F3C81930F9195CC
:104650003D81931731F080E993E00E94BD2B84E007
:104660000EC090E00596080F191F27FFDECFF70157
:104670001183008380E003C083E001C081E02896BD
:104680000FB6F894DEBF0FBECDBFDF91CF911F9163
:104690000F91FF90EF9008959F92AF92BF92CF92AB
:1046A000DF92EF92FF920F931F93CF93DF93CDB7DB
:1046B000DEB7C850D1400FB6F894DEBF0FBECDBFF5
:1046C0006C01962E5A01FC01108280E560E070E0DA
:1046D00048E050E09E012F5F3F4F0E9481228823D7
:1046E00009F06DC0FE01319697E02191820F915043
:1046F000E1F781959885891709F05BC00E8110E07C
:1047000093E0000F111F9A95E1F70115110509F4C7
:1047100052C080E5B80145E050E09E012F5F3F4F59
:104720000E948122882309F04AC08A819981890FD9
:10473000EB808E0D9C81890F81959D818917E9F50C
:10474000FF240B5F1F4F80E5B801A7019E01275F83
:104750003F4F0E948122882391F590E00AC049E0F2
:1047600050E04C0F5D1F240F351FF9012081920F7F
:104770008F5F282F30E02E153F0588F391958C81AF
:104780009817F9F4F60180818F5F8083891559F4B9
:10479000A114B10441F0F501DE0119968DE00D90F0
:1047A00001928150E1F78A8187FD0DC00E0D1F1D1A
:1047B000B0CF82E009C083E007C084E005C081E09B
:1047C00003C085E001C080E0C85FDE4F0FB6F894FB
:1047D000DEBF0FBECDBFDF91CF911F910F91FF9034
:1047E000EF90DF90CF90BF90AF909F9008957F9211
:1047F0008F929F92AF92BF92CF92DF92EF92FF92F1
:104800000F931F93CF93DF93CDB7DEB7A1970FB66A
:10481000F894DEBF0FBECDBF85E78B8384E48C8325
:1048200087E58D8383E48E831092E90332E0E32EE3
:10483000F12CEC0EFD1EC70160E040E050E00E944C
:10484000DA0A5E010894A11CB11CC50160E040E0D9
:1048500050E00E944C238A81882319F489E890E172
:1048600006C08981882309F07DC082EA90E10E9418
:10487000CF2B11E08CC0872D982D6D2DAE014C5E95
:104880005F4F0E94DA0A8BEB90E10E94CF2B8E01E2
:104890000C5E1F4F20E0F80181918F0129A30E9437
:1048A000482C8DEA93E00E94BD2B29A12F5F2D306B
:1048B00091F788E793E00E94BD2B11E001E0AA2464
:1048C000A3944AC0892D9C2D602FAE01495F5F4F94
:1048D0000E944C238A85803351F5112341F186ECE7
:1048E00090E10E94CF2B27E0E22EF12CEC0EFD1E72
:1048F00010E0F70181917F010E94482C8DEA93E03E
:104900000E94BD2B1F5F1D30A1F788E793E00E9436
:10491000BD2BCE014796BE01665F7F4F4AE050E057
:104920000E946F2F009711F011E001C010E08A85FE
:10493000823389F48091E903882369F4CE010396D8
:10494000BE01645F7F4F44E050E00E946F2F0097EC
:1049500011F4A092E9030F5F8981801708F0B2CFAC
:10496000D39407C011E0DD24D3947E2C8F2C9A2C95
:10497000CB2C8A818D1518F0112309F07CCF91E0A2
:10498000111190E08091E90389238093E903812F3D
:10499000A1960FB6F894DEBF0FBECDBFDF91CF91C9
:1049A0001F910F91FF90EF90DF90CF90BF90AF904D
:1049B0009F908F907F9008950F931F93CF93DF93D5
:1049C00000D0CDB7DEB7062F142F7A8389830E94DB
:1049D00063298981880F0E9486297A81882351F072
:1049E000872F0E948629882329F0802F0E948629FC
:1049F000882321F40E947B2981E00CC0812F0E9432
:104A000086290E947B298FE097E20197F1F700C089
:104A1000000080E00F900F90DF91CF911F910F91D8
:104A20000895AF92BF92CF92DF92EF92FF921F93C1
:104A3000CF93DF93182F6B015A017901C0E0D0E0CA
:104A40000AC0F70141917F01BE016C0D7D1D812FD0
:104A50000E94DC242196CA15DB0599F780E0DF91DE
:104A6000CF911F91FF90EF90DF90CF90BF90AF90CC
:104A70000895AF92BF92CF92DF92EF92FF920F9381
:104A80001F93CF93DF930F92CDB7DEB7082F6A0144
:104A9000E22EA32E69830E946329802F880F0E9433
:104AA000862969818823B9F0862F0E948629882368
:104AB00091F00E946E29802F880F81600E948629C4
:104AC000882349F00E2D1A2DEE24FF245601089458
:104AD000A108B10813C00E947B2981E015C0EA1427
:104AE000FB0411F480E001C081E00E94BC29F801C0
:104AF00080830894E11CF11C0F5F1F4FEC14FD0430
:104B000071F70E947B2980E00F90DF91CF911F9178
:104B10000F91FF90EF90DF90CF90BF90AF900895EE
:104B2000CF92DF92EF92FF920F931F93CF93DF9379
:104B300000D0CDB7DEB77A0169016A8389830E940C
:104B400063298981880F0E9486296A81882381F0E0
:104B5000862F0E948629882359F08601CC24DD24E3
:104B60000EC0F80181918F010E948629882321F4CB
:104B70000E947B2981E00FC00894C11CD11CCE1477
:104B8000DF0479F70E947B298FE097E20197F1F724
:104B900000C0000080E00F900F90DF91CF911F9137
:104BA0000F91FF90EF90DF90CF9008950F931F9398
:104BB000CF93DF9300D0CDB7DEB78A016A838983B4
:104BC0000E9463298981880F0E9486296A8188232F
:104BD000E1F0862F83700E9486298823B1F0F801C6
:104BE00080810E948629882381F0F80181810E94BA
:104BF0008629882351F00E947B298FE097E2019754
:104C0000F1F700C0000080E003C00E947B2981E032
:104C10000F900F90DF91CF911F910F910895CF9238
:104C2000DF92EF92FF928091B7038093B6032091B9
:104C3000F3032093B7038091F203882389F0309126
:104C400017068091F0039091F10330FF03C08D7F30
:104C5000816002C082608E7F9093F1038093F003A5
:104C6000233009F467C1243048F48091B603213021
:104C700009F4A1C0223008F023C10DC0253009F489
:104C8000E7C1253008F460C1263009F42DC22B306D
:104C900009F057C264C0882389F180E490E09093C2
:104CA000F1038093F003469883E69EE00E94CF2BA9
:104CB00080E79EE00E94CF2B8091F1030E94482C58
:104CC0008091F0030E94482C88E793E00E94BD2B5E
:104CD0000E94FC291092FA0380E060E040E020E0AE
:104CE0000E942A2081E060E040E020E00E942A202B
:104CF00082E060E040E020E00E942A201092F2036F
:104D000035992AC00E94092B882329F08091FA0343
:104D10008F5F8093FA038091FA03843608F411C2FE
:104D20000E944D29882321F48BE79EE00E94CF2B1F
:104D30001092FA038091F0039091F1038F7B8062CF
:104D40009093F1038093F00380E061E040E020E085
:104D50000E942A208BE0F3C11092FA03F2C18091E5
:104D6000BF05882309F4EDC18EE99EE00E94CF2B98
:104D7000C090E103D090E203E090E303F090E403FD
:104D80000E94F7238093FB038091E1039091E2035B
:104D90008C199D090E94FF2B89EB9EE00E94CF2B6E
:104DA0000E94F82985E00E94752081E08093F3033A
:104DB0008093EA03C6C1813009F444C08DEB9EE0C4
:104DC0000E94CF2B8091B6038B3069F58091FB0355
:104DD000882399F48AEC9EE00E94CF2B87E00E9402
:104DE00075208091F0039091F10380689093F10316
:104DF0008093F00381E060E012C080EE9EE00E94AC
:104E0000CF2B88E00E9475208091F0039091F103F0
:104E100091609093F1038093F00381E061E040E0C2
:104E200020E00E942A208FEF9EE00E94CF2B8091ED
:104E3000F1030E94482C8091F0030E94482C8AE0E4
:104E40009FE07FC08091F00387FF35C08091BF0550
:104E5000882389F18091F203882361F00E94BF20AA
:104E6000882341F08CE09FE00E94CF2B80E00E94DD
:104E7000752015C08091F2038823A1F08091EA0388
:104E8000882381F08091170680FD0CC086E29FE0A8
:104E90000E94CF2B80E00E9475201092EA0382E0EE
:104EA0008093F3038091EF03882329F084E08093BB
:104EB000F3031092EF03359B44C184E49FE036C1B5
:104EC0008230A1F089E59FE00E94CF2B86E69FE02B
:104ED0000E94CF2B8091F1030E94482C8091F00317
:104EE0000E94482C88E793E00E94BD2B0E94D120AD
:104EF000882351F081E79FE00E94CF2B81E00E9440
:104F0000752081E08093F303359B09C085E89FE01D
:104F10000E94CF2B86E00E9475201092F3038091AF
:104F2000EF03882309F40DC184E08093F30310920A
:104F3000EF0307C18091B603833009F402C18AE907
:104F40009FE00E94CF2BFDC08091B603843071F1A9
:104F50008091F0039091F1038B7F9093F103809304
:104F6000F00387EA9FE00E94CF2B84EB9FE00E9432
:104F7000CF2B8091F1030E94482C8091F0030E9476
:104F8000482C88E793E00E94BD2B469A1092FA03C2
:104F90008091E903882351F08CE061E043EB53E01A
:104FA0000E94D6258FEB9FE00E94CF2B0E94092BF9
:104FB000882339F08091FA038F3118F48F5F809342
:104FC000FA038091FA038E3159F48CE760E040E4F3
:104FD0000E94D72182E061E040E020E00E942A2088
:104FE0000E94D1208823A1F08091F0039091F103D9
:104FF00082608E7F9093F1038093F0038AED9FE0AF
:105000000E94CF2B81E00E94752085E08093F303FE
:105010008091ED03882319F085E08093F303359B9D
:1050200090C08EEE9FE00E94CF2B86E00E947520FC
:105030008091E903882309F47EC08CE061E04FEAA7
:1050400053E00E94D62583E090E10E94CF2B73C0ED
:105050008091B603853041F189E190E10E94CF2B28
:1050600086E290E10E94CF2B8091F1030E94482CB0
:105070008091F0030E94482C88E793E00E94BD2BAA
:1050800082E060E040E020E00E942A208091E90375
:10509000882351F08CE061E04FEA53E00E94D6256E
:1050A00081E390E10E94CF2B8091ED03882371F082
:1050B0008091F0039091F10384609093F1038093C9
:1050C000F00382E00E9475201092ED038091EE03C0
:1050D000882329F086E08093F3031092EE03359B3A
:1050E00030C087E490E122C08091B6038630D1F0D1
:1050F0008CE760E440E40E94D72146988CE590E17B
:105100000E94CF2B89E690E10E94CF2B8091F10382
:105110000E94482C8091F0030E94482C88E793E07D
:105120000E94BD2B359B0AC084E790E10E94CF2BE3
:1051300086E00E9475201092F30303C081E0809303
:10514000F3038091EB03882331F08091B5030E9433
:1051500075201092EB03FF90EF90DF90CF900895B1
:10516000EF92FF921F93CF93DF930F92CDB7DEB7ED
:10517000182F7A0169830E946329812F880F0E946A
:10518000862969818823E9F0862F83700E94862909
:105190008823B9F00E946E29812F880F81600E94B8
:1051A0008629882371F081E00E94BC29F701808361
:1051B00080E00E94BC29F70181830E947B2980E066
:1051C00003C00E947B2981E00F90DF91CF911F9156
:1051D000FF90EF900895CF93DF9300D0CDB7DEB767
:1051E0006A8389830E9463298981880F0E948629A6
:1051F0006A81882329F0862F0E948629882321F43A
:105200000E947B2981E009C00E947B298FE097E200
:105210000197F1F700C0000080E00F900F90DF9140
:10522000CF910895CF92DF92EF92FF920F931F9349
:10523000CF93DF930F92CDB7DEB77B0189830E94B6
:1052400063298981880F81600E948629882321F43F
:105250000E947B298FEF17C081E00E94BC29182F84
:1052600000E080E00E94BC29C82EDD24C02AD12A9B
:105270000E947B29E114F10411F48D2D04C0F70183
:10528000D182C08280E00F90DF91CF911F910F916A
:10529000FF90EF90DF90CF9008958BB18F7C8BB90A
:1052A0008AB18F7C8AB989E096E09A95F1F700C0BF
:1052B000549A96E09A95F1F700C054988150A1F75E
:1052C00089B180720895559A86E08A95F1F700C0F9
:1052D000549A86E08A95F1F700C00895559886E0C3
:1052E0008A95F1F700C0549886E08A95F1F700C0DE
:1052F0000E9463290895549886E08A95F1F700C0CA
:10530000559886E08A95F1F700C00895F89428E052
:1053100030E090E8492F482311F4559A01C0559880
:1053200046E04A95F1F700C054984DE04A95F1F7F0
:105330000000549A46E04A95F1F700C09695215036
:10534000304041F7559886E08A95F1F700C05498AF
:1053500046E04A95F1F700C099B186E08A95F1F7E9
:1053600000C0549A559A46E04A95F1F700C07894E7
:1053700081E095FD80E00895282FF894559898E0F5
:1053800080E0880F36E03A95F1F700C0549836E097
:105390003A95F1F700C04D99816036E03A95F1F702
:1053A00000C0549A36E03A95F1F700C0915049F7A1
:1053B000222311F0559A01C0559896E09A95F1F77D
:1053C00000C054983DE03A95F1F70000549A559A80
:1053D00096E09A95F1F700C0789408958091FE03C5
:1053E000882319F08BE090E0089589E090E008951B
:1053F00081E08093FE0308951092FE0308958BB11F
:105400008F738BB98AB18F738AB90895579A86E0E2
:105410008A95F1F700C0569A86E08A95F1F700C0A8
:105420000895579886E08A95F1F700C0569886E06F
:105430008A95F1F700C00E94062A0895569886E0E2
:105440008A95F1F700C0579886E08A95F1F700C079
:10545000089528E030E090E8492F482311F4579A46
:1054600001C0579846E04A95F1F700C056984DE0C4
:105470004A95F1F70000569A46E04A95F1F700C0C8
:1054800096952150304041F7579886E08A95F1F77C
:1054900000C0569896E09A95F1F700C089B146E0B1
:1054A0004A95F1F700C0569A579A96E09A95F1F707
:1054B00000C08095881F8827881F0895282F579837
:1054C00098E080E0880F36E03A95F1F700C05698F2
:1054D00036E03A95F1F700C04F99816036E03A9591
:1054E000F1F700C0569A36E03A95F1F700C09150B6
:1054F00049F7222311F0579A01C0579896E09A95E0
:10550000F1F700C056983DE03A95F1F70000569A41
:10551000579A96E09A95F1F700C008959091350654
:1055200083B1809589279091FF039823909590935C
:10553000FF032091000428232927209300049823A7
:105540009223809135068927809335062091340671
:10555000809135068923822B80933406209133066F
:105560008091350680958923822B80933306089598
:10557000F89490913406892390913406982790935B
:10558000340678940895F894909133068923909185
:10559000330698279093330678940895F894909161
:1055A00035067894892308958093050481E08093DB
:1055B0000404089510920404089581E09091040475
:1055C000992309F480E0089580910504882329F047
:1055D00081508093050480E0089581E008958093D0
:1055E000030481E080930204089510920204089558
:1055F00081E090910204992309F480E0089581E00C
:1056000090910304911180E0089581E0809301045A
:10561000089580910104882321F01092010481E013
:10562000089580E008951092C5008CE08093C40036
:1056300088E98093C1001092B8061092B6061092C5
:10564000B7061092390708959091B6062091B806D2
:1056500091509F772917C1F3E091B806F0E0E75425
:10566000F94F80838091B8068F5F8093B806809150
:10567000B806803811F41092B8068091C10080629B
:105680008093C10008953091B706209139073217F1
:10569000A1F020913907E22FF0E0EA5CF94F308168
:1056A000FC0130832F5F20933907809139078038C0
:1056B00031F41092390780E0089581E0089580E088
:1056C00008951F920F920FB60F920BB60F921124EE
:1056D0008F939F93EF93FF93E091B606F0E0E7542A
:1056E000F94F80818093C6008091B6068F5F8093CA
:1056F000B6068091B606803811F41092B6069091E5
:10570000B8068091B606981729F48091C1008F7D64
:105710008093C100FF91EF919F918F910F900BBEED
:105720000F900FBE0F901F9018951F920F920FB6FB
:105730000F920BB60F9211248F939F93EF93FF93C9
:105740008091B706E82FF0E09091C600EA5CF94F2F
:1057500090838F5F8093B7068091B706803811F4ED
:105760001092B706FF91EF919F918F910F900BBE12
:105770000F900FBE0F901F901895CF93DF93EC0101
:1057800008C08A3019F48DE00E94242B89910E9470
:10579000242B88818823A9F7DF91CF9108951F9347
:1057A000CF93DF93EC012196FC0114911A3019F488
:1057B0008DE00E94242B812F0E94242BFE01219634
:1057C0001491112399F7DF91CF911F9108950F93B1
:1057D0001F93CF93DF93082FC8E0D0E010E8812F0C
:1057E000802311F081E301C080E30E94242B1695F1
:1057F0002197A9F7DF91CF911F910F910895DF9223
:10580000EF92FF920F931F93CF93DF93CDB7DEB745
:1058100029970FB6F894DEBF0FBECDBF8C01DE0115
:105820001196E8EBF3E088E001900D928150E1F7EA
:105830007E010894E11CF11C84E0D82E91E010C098
:105840008F5F021B130B90E002171307C8F7992311
:1058500029F4805D99870E94242B9985DA9431F090
:10586000F701219131917F0180E0EECF802F805DA3
:105870000E94242B29960FB6F894DEBF0FBECDBF31
:10588000DF91CF911F910F91FF90EF90DF900895DE
:105890001F93CF93DF93CDB7DEB760970FB6F89421
:1058A000DEBF0FBECDBF182FDE011196E0ECF3E096
:1058B00080E101900D928150E1F7812F82958F70E8
:1058C000E1E0F0E0EC0FFD1FE80FF11D80810E9488
:1058D000242B1F70E1E0F0E0EC0FFD1FE10FF11D44
:1058E00080810E94242B60960FB6F894DEBF0FBE15
:1058F000CDBFDF91CF911F910895CF93DF93CDB7A7
:10590000DEB7C354D0400FB6F894DEBF0FBECDBF94
:105910001092BF0580E880BFA89528E288E190E05A
:105920000FB6F894A895809360000FBE2093600096
:105930001092C3051092C4051092C5051092C605B9
:105940001092C9050E94132B0E9493080E94FF2900
:105950000E9422209093CE058093CD0589E080930C
:1059600081008FE39FE1909389008093880082E01B
:1059700080936F002C9885B1806685B984B180676B
:1059800084B94098389A139A149881B1886181B982
:1059900015980D9A46983E9A5A9A5B9880E060E175
:1059A0004FE154E027E234E00E94FF1081E060E222
:1059B0004FE054E027E334E00E94FF1082E060E40F
:1059C00047E154E02FE234E00E94FF101092C70537
:1059D00078948FEF9FE00E94952F082F8F3F31F42E
:1059E0008FEF9FE060E00E94A72F00E080EE93E041
:1059F0000E94CF2B88EF93E00E94CF2B802F0E9434
:105A0000482C87E094E00E94CF2B82B18C7F82B932
:105A100000FD119A01FD109A1092C2058BE193E0EE
:105A20000E94BD2B0E94B40E0E94FF2B89E094E0DF
:105A30000E94CF2B8BE094E00E94CF2B80916000DE
:105A40000E94482C84E194E00E94CF2B86E194E0F0
:105A50000E94CF2B82E393E00E94BD2B8FE194E064
:105A60000E94CF2B85E394E00E94CF2B8BE394E040
:105A70000E94CF2B8BE494E00E94CF2B81E594E031
:105A80000E94CF2B8CE594E00E94CF2B85E694E01A
:105A90000E94CF2B8AE694E00E94CF2B86E794E009
:105AA0000E94CF2B8AE794E00E94CF2B83E894E0FA
:105AB0000E94CF2B85E894E00E94CF2B84B70E94F0
:105AC000482C8DE894E00E94CF2B14BE0E94D11385
:105AD0008093C8050E94570F88E393E00E94BD2B76
:105AE0008091C8050E94482C89E493E00E94BD2B58
:105AF0000E941F0E80E2809313061092140600E0AD
:105B000010E0FF24FA94A8950E94580E0E945B09A9
:105B10008091BD058823B1F080E96AEB75E00E94B1
:105B20002C1382E960EC75E00E942C130E94EE2990
:105B30008A30910528F088E46BEC75E00E94122908
:105B40001092BD050E940F268091BE05882321F08A
:105B50000E942F211092BE050E94670F882311F02A
:105B6000A895FACF0E94D70F8091CD059091CE05D0
:105B7000FC01208120FF2AC00E944614E091CD053F
:105B8000F091CE0590819E7F90838823F9F4CF0118
:105B90000E9413142091CD053091CE05882389F4FD
:105BA000C901BE016F5F7F4F0E946D14882371F0A1
:105BB000CE0101960E941914CE0101960E94DB10BD
:105BC00005C0C9010E9425200E94F9108091CA05D4
:105BD000882309F498CF0E94DD2A882379F00E9457
:105BE000E42A882359F081E08093C7050E94DA2ACD
:105BF0008FE894E00E94CF2B00E010E08091C30575
:105C00009091C405A091C505B091C6050196A11D4E
:105C1000B11D8093C3059093C405A093C505B093AF
:105C2000C60580E00E94B61181E00E94B61182E0B4
:105C30000E94B6118091C705843009F460C0853098
:105C400040F48130E9F0813070F0833009F0A2C077
:105C500037C0863009F48CC0863008F471C08730B4
:105C600009F098C087C081B18C7F81B98AB1837FE8
:105C70008AB90D9A389A139A14981092C9058AC055
:105C800080E00E940709F2E08C3B9F0708F482C085
:105C90000F5F1F4F0230110509F07CC083E0809335
:105CA000C7051398149A89EA94E00E94CF2B80913B
:105CB000C3059091C4050E94FF2B82ED94E01CC0A7
:105CC0000530110519F481B1836081B90F5F1F4F51
:105CD0000531110508F45EC0389884E08093C7054B
:105CE00085ED94E00E94CF2B8091C3059091C4056F
:105CF0000E94FF2B85E095E00E94CF2B49C0319B8D
:105D000049C081E08093BF050F5F1F4F063011052A
:105D100008F440C00D988AB18C608AB985E0809300
:105D2000C70588E095E00E94CF2B8091C305909134
:105D3000C4050E94FF2B86E395E00E94CF2B2AC06A
:105D40008091C905882331F589E395E00E94CF2B26
:105D50008091C3059091C4050E94FF2B8CE495E0CF
:105D60000E94CF2B0E94EA0E81E08093C90512C0E9
:105D70000D9A10C0389A0D9A8AB1837F8AB9139A06
:105D8000149881E08093C2051092C7051092C9054E
:105D900000E010E0E090C705FE1409F441C022E0E5
:105DA000E216B9F02E1530F081E0EE2071F0E81621
:105DB000B9F50AC0E5E0EE16E1F0F7E0EF1621F1E3
:105DC00024E0E21669F50AC081E060E041E050E0BD
:105DD0001FC081E060E042E050E01AC081E060E076
:105DE00040E050E00E94191182E060E042E050E0A3
:105DF00015C081E060E040E050E00E94191182E0AF
:105E000060E041E050E00AC081E060E040E050E046
:105E10000E94191182E060E040E050E00E941911F8
:105E20001092CA05FE2C6FCE629FD001739FF001C5
:105E3000829FE00DF11D649FE00DF11D929FF00D1A
:105E4000839FF00D749FF00D659FF00D9927729F51
:105E5000B00DE11DF91F639FB00DE11DF91FBD01DC
:105E6000CF0111240895991B79E004C0991F96175A
:105E700008F0961B881F7A95C9F78095089597FBBF
:105E8000092E07260AD077FD04D00CD006D00020BA
:105E90001AF4709561957F4F0895F6F79095819566
:105EA0009F4F0895AA1BBB1B51E107C0AA1FBB1F30
:105EB000A617B70710F0A61BB70B881F991F5A9596
:105EC000A9F780959095BC01CD010895FB01DC01F7
:105ED00002C005900D9241505040D8F70895FB0143
:105EE000DC0104C08D910190801921F44150504093
:105EF000C8F7881B990B0895FB01DC0102C00190D3
:105F00000D9241505040D8F70895DC01CB01FC01BF
:105F1000F999FECF06C0F2BDE1BDF89A319600B402
:105F20000D9241505040B8F70895F999FECF92BDB7
:105F300081BDF89A992780B50895DC01CB0103C093
:105F40002D910E94A82F41505040D0F70895262F40
:105F5000F999FECF1FBA92BD81BD20BD0FB6F8944E
:0E5F6000FA9AF99A0FBE01960895F894FFCFB1
:105F6E000A0001FFFF204552524F5221003A2030C5
:105F7E0078000A002E2E2E204552524F52210A0032
:105F8E002E2E2E20646F6E65210A00646F6E6521C1
:105F9E000A00205265616420556E697175652D4940
:105FAE00443A200020525F4552524F522100206D3C
:105FBE00560A0020000A0A383330303E0A00756E49
:105FCE006B6E6F776E20636F6D6D616E640A003855
:105FDE003330303E00535441540048454C5000522B
:105FEE00544D310052544D320052544D33005254E0
:105FFE004D340052544D350052544D360052544DCE
:10600E00370052544D3800564F4C540050524F4D9D
:10601E000049440044414357004441435200007537
:10602E0002D30D7A02E70B7F02AC0D8402850D8937
:10603E0002730D8E026A0D9302610D9802580D9D2A
:10604E0002E10BA202190DA702C30CAC02670CB140
:10605E0002810CB402180CB902ED0BBE0200000A4C
:10606E0000726571206F75742064726F7070656454
:10607E0020616674657220330A000A4D6F64756C78
:10608E00652053657269616C204E756D6265723A5A
:10609E002000322E372E32004D6F64756C65204114
:1060AE006464726573733A20000A0A000A006F6610
:1060BE0066733A0020636E743A002000322E372E3B
:1060CE00320044062A069B07EA055B071B07DB0620
:1060DE00AA056A059B065B060A0072746D20636D45
:1060EE006E206864722063686B206661696C0A00BA
:1060FE006D756C7420686561646572206368656394
:10610E006B73756D206572726F72210A002000200C
:10611E00002FFC2C1C06FFFF1027E80364000A006A
:10612E0030313233343536373839414243444546BF
:00000001FF
